:1000000017C03BC03AC039C039C237C036C035C04E
:1000100034C033C032C031C030C02FC02EC0003712
:1000200000380101010101010102040810208502CC
:1000300011241FBECFE5D2E0DEBFCDBF10E0A0E6A9
:10004000B0E0E2E6F7E002C005900D92AA37B107F2
:10005000D9F720E0AAE7B0E001C01D92A939B207A4
:10006000E1F710E0C8E1D0E003C02197FE0171D3B1
:10007000C731D107D1F773D272C3C2CF282F30E076
:10008000F901E85DFF4F9491F901EE5DFF4FE491B6
:10009000EE23A1F0811113C08AB58F738ABDF0E001
:1000A000E05EFF4FA491B0E08FB7611113C0F894E8
:1000B0002C91E92FE095E223EC938FBF08958130D6
:1000C00019F48AB58F7CEACF843049F78CB58F7CE0
:1000D0008CBDE5CFF894EC91E92BEECF3FB7F894C7
:1000E00080917F0090918000A0918100B09182006A
:1000F0002FB508B602FE05C02F3F19F00196A11DCD
:10010000B11D3FBFBA2FA92F982F8827BC01CD0161
:10011000620F711D811D911D42E0660F771F881FC0
:10012000991F4A95D1F70895CF92DF92EF92FF92EF
:10013000CF93DF936B017C01D1DFEB01C114D104BC
:10014000E104F10439F4DF91CF91FF90EF90DF905B
:10015000CF900895C3DF6C1B7D0B683E734070F336
:1001600081E0C81AD108E108F108C851DC4FE6CF98
:100170004F925F926F927F928F929F92AF92BF92B7
:10018000CF92DF92EF92FF920F931F93CF93DF9363
:10019000F82E60918A00681B770B77FF03C071957A
:1001A00061957109072E000C880B990B20918E0028
:1001B00030918F0050E040E061D22CE330E040E02D
:1001C00050E091D28091900090919100B0E0A0E039
:1001D000281739074A075B0760F0809192009091D9
:1001E0009300B0E0A0E0281739074A075B0708F43E
:1001F000C901EC0110918D002F2D1F1508F4212F3E
:1002000020938A00C0909600D09097002601712C10
:10021000612CE0909400F09095004701B12CA12C46
:10022000C301B601681979098A099B0930E050E0D9
:1002300040E024D2212F30E050E040E038D2DA0113
:10024000C901880D991DAA1DBB1D88159905AA0510
:10025000BB053CF07C01481659066A067B060CF487
:100260007601F0928C00E0928B00F12CE12C08EEEC
:1002700013E0EC16FD0608F043C061E080918900B0
:10028000FDDE80918B0090918C008E7F0097D9F4D9
:1002900060E080918900F2DE209731F06091980053
:1002A00070E090E080E040DF80918B0090918C00C6
:1002B000B8013BD280919800680F711D6F5F7F4F2E
:1002C000E60EF71ED6CF0000000000000000000080
:1002D000000000000000000000000000000000001E
:1002E000000000000000000000000000000000000E
:1002F0000000000000000000000000000297C6CFD0
:10030000DF91CF911F910F91FF90EF90DF90CF90F1
:10031000BF90AF909F908F907F906F905F904F9025
:10032000089508958FEF9FEF089590E080E008957D
:10033000CF92DF92EF92FF920F931F93CF93DF93B1
:100340006C01EB017B01E40EF51E10E000E0CE1520
:10035000DF0561F06991D601ED91FC910190F0818A
:10036000E02DC6010995080F191FF1CFC801DF91D3
:10037000CF911F910F91FF90EF90DF90CF90089554
:10038000DC0114968D919C91DC01ED91FC91028031
:10039000F381E02D099581E090E00895682F83E8CE
:1003A00090E0EECF08954F925F926F927F92AF925E
:1003B000BF92CF92DF92EF92FF921F93CF93DF9382
:1003C000CDB7DEB7A1970FB6F894DEBF0FBECDBF95
:1003D0006B017C01B12CA12CF7FE0BC08DE2DEDF9E
:1003E0005C01F094E094D094C094C11CD11CE11C39
:1003F000F11C1C2D7D2DC70119A27E0121E2E20E08
:10040000F11C2AE0422E512C612C712C612FA3018A
:10041000920169D1822F6AE028D1181B1A3064F545
:10042000105DF70112937F01122F732FCA01232B46
:10043000242B252B59F701900020E9F73197AF01C4
:100440004E195F09B70183E890E072DF8A0D9B1DAA
:10045000A1960FB6F894DEBF0FBECDBFDF91CF914E
:100460001F91FF90EF90DF90CF90BF90AF907F9063
:100470006F905F904F900895195CD3CF78941F923E
:100480000F920FB60F9211242F933F938F939F9348
:10049000AF93BF9380917B0090917C00A0917D00F1
:1004A000B0917E0030917A002CE7230F2D3728F091
:1004B0002FEF230F0196A11DB11D20937A00809389
:1004C0007B0090937C00A0937D00B0937E00809190
:1004D0007F0090918000A0918100B09182000196F0
:1004E000A11DB11D80937F0090938000A093810097
:1004F000B0938200BF91AF919F918F913F912F91C7
:100500000F900FBE0F901F901895E3E8F0E0138254
:1005100012828EE690E09183808380E690E095835E
:100520008483E9E8F0E08FEF808381831382128275
:1005300084EB848386EE90E0968385831086178211
:100540008FEF9FEF928781878CEB92E09487838770
:100550008CEF98E09687858780E187870895789467
:1005600080B7806880BF80B7806480BF8CB58064AE
:100570008CBD9FEF9DBD80B7807F876080BF89B7AE
:10058000846089BF83B7887F83BF8AB58C7F816091
:100590008ABD83B7877F83BF83B7887F836083BF2C
:1005A00086B1876086B9379A81E0809389009093FD
:1005B0008A0010928C0010928B00E9E2F0E0249106
:1005C000E3E2F0E0E491EE2389F08E2F90E0FC016D
:1005D000E25EFF4FA491B0E0805E9F4FFC018491EA
:1005E0008FB7F894EC91E22BEC938FBF60E0809191
:1005F000890044DDC12CD12C76018C2DB9DDC701D9
:10060000B601D1DE8DE0CADE8AE0C8DE64E170E0CA
:1006100080E090E089DDFFEFCF1ADF0AEF0AFF0AE2
:1006200085EBC816D104E104F10439F784EBC82E38
:10063000D12CE12CF12C8C2D9BDDC701B601B3DE52
:100640008DE0ACDE8AE0AADE64E170E080E090E05C
:100650006BDDE1E0CE1AD108E108F108FFEFCF161B
:10066000DF06EF06FF0639F7C5CF002480FD060E32
:10067000660F11F08695D1F7802D0895EE27FF279C
:10068000AA27BB2708C0A20FB31FE41FF51F220F24
:10069000331F441F551F969587957795679598F357
:1006A0007040A9F7009799F7BD01CF010895052E75
:1006B00097FB16F400940FD057FD05D014D007FC1B
:1006C00002D046F408C050954095309521953F4F93
:1006D0004F4F5F4F089590958095709561957F4F2E
:1006E0008F4F9F4F0895A1E21A2EAA1BBB1BFD013D
:1006F0000DC0AA1FBB1FEE1FFF1FA217B307E40701
:10070000F50720F0A21BB30BE40BF50B661F771F58
:10071000881F991F1A9469F7609570958095909538
:100720009B01AC01BD01CF010895AA1BBB1B51E188
:1007300007C0AA1FBB1FA617B70710F0A61BB70B51
:10074000881F991F5A95A9F780959095BC01CD01F6
:100750000895EE0FFF1F0590F491E02D0994F89491
:02076000FFCFC9
:100762006600000000009101D20100000000C001FB
:0A0772009801950192019201910196
:00000001FF
